:100000008312031385010528642F07309F00831690
:100010008E15F030850086018312FF308100FD01CE
:10002000F4018030FF000515851405140B118B16A3
:100030008B17F301F401F501F201E801E901E40194
:100040007308E5007408E6007508E7006508031901
:100050000C30E400F6306407031C3528E400583007
:10006000F000A830F10058307E214430F000BC3060
:10007000F1006C30E408031D3F280E216028E40BDA
:1000800043287E216028E40B4728B7216028E40B31
:100090004B2806226028E40B4F2862226028E40BDC
:1000A0005328BD226028E40B57281B236028E40B4B
:1000B0005B2884236028E40B5F28C523602846243E
:1000C0003030F000D030F10080305E251C30F00080
:1000D000E430F1006608E400F630E4070318732802
:1000E00094300E218E28E4070318792894307E215D
:1000F0008E28E40703187F289430B7218E28E40760
:1001000003188528943006228E28E40703188B28CC
:10011000943062228E28E4079430BD220A30E4072E
:100120000830F000F830F100A830E408031D9A28E8
:100130000E21BB28E40B9E287E21BB28E40BA228BD
:10014000B721BB28E40BA6280622BB28E40BAA286B
:100150006222BB28E40BAE28BD22BB28E40BB228E8
:100160001B23BB28E40BB6288423BB28E40BBA2846
:10017000C523BB284624F430F0000C30F100BC301D
:100180006318C4280C25C528AF24F001F101803084
:10019000AC256608FD008030EE00EF000530EB0076
:1001A0001E30EC00C426650DFD007D0DFC39650791
:1001B000FD00660CFE007E0C3F39FE00FD30FE07A0
:1001C000031CE428FD0ADE288030EE00EF00083032
:1001D000EB000F30EC00B6266708FD008030EE0023
:1001E0004030EF000830EC00AC2685110000F62806
:1001F0008600051005110515700708008600051416
:10020000051105158510851471070800E2001830E6
:10021000FF3E031808296208851508008511F8209B
:100220000A3EFE200621F43EF8200B3EFE20F33E5F
:10023000F8200C3EFE20F33EF8200B3EFE20F43E5C
:10024000F8200A3EFE20F63EF820073EFE20F93E4A
:10025000F820043EFE20FD3EF820013EFE20F8205E
:10026000FE3EFE20043EF820FB3EFE20073EF82026
:10027000F83EFE200A3EF820F73EFE200B3EF82016
:10028000F63EFE200B3EF820F73EFE200A3EF82008
:10029000F83EFE20083EF820FB3EFE20053EF820FA
:1002A000FE3EFE20013EF820013EFE20FE3EF820EC
:1002B000043EFE20FA3EF820073EFE20F73EF820DE
:1002C0000A3EFE20FC3EF820043EFE20FA3EF820C6
:1002D000033EFE20FB3EF820023EFE20FC3EF820BE
:1002E000013EFE20FD3EF820FE20FE3EF820FF3EAF
:1002F000FE20FF3EF820FE3EFE2008008511FC3E59
:10030000F8200A3EFE200621F73EF8200A3EFE2095
:10031000F73EF8200A3EFE20F73EF8200A3EFE2077
:10032000F73EF8200A3EFE20F63EF820083EFE206A
:10033000F83EF820063EFE20FA3EF820043EFE205D
:10034000FC3EF820023EFE20FE3EF820FE20F82073
:10035000FE3EFE20023EF820FC3EFE20043EF82039
:10036000FA3EFE20063EF820F83EFE2008008511E9
:10037000FA3EF8200E3EFE200621F43EF8200D3E07
:10038000FE20F53EF8200C3EFE20F63EF8200A3E08
:10039000FE20F83EF820083EFE20FA3EF820053EFA
:1003A000FE20FD3EF820023EFE20FE3EF820FE200C
:1003B000F820FE3EFE20F820FE3EFE20F820FE3E05
:1003C000FE20F820FE3EFE20F820FE3EFE20F82013
:1003D000FE3EFE20F820FE3EFE20043EF820FC3EBD
:1003E000FE20063EF820FA3EFE20083EF820F83EA9
:1003F000FE200A3EF820F63EFE200C3EF820F43E99
:10040000FE200E3EF820F23EFE2008008511FA3E46
:10041000F8200E3EFE200621F43EF8200D3EFE2080
:10042000F53EF8200C3EFE20F63EF8200A3EFE2067
:10043000F83EF820083EFE20FA3EF820053EFE2059
:10044000FD3EF820023EFE20FE3EF820FE20F82071
:10045000FE3EFE20F820FF3EFE20FF3EF820FE205C
:10046000FE3EF820023EFE20F820FE20023EF8204C
:10047000FD3EFE20053EF820FA3EFE20063EF82016
:10048000F83EFE20083EF820F63EFE200A3EF82008
:10049000F43EFE200A3EF820F53EFE20093EF820FC
:1004A000F63EFE20083EF820F83EFE20063EF820EC
:1004B000FA3EFE20043EF820FD3EFE20013EF820DC
:1004C000FE2008008511023EF820F63EFE2006219F
:1004D0000A3EF820F83EFE20083EF820FA3EFE20B4
:1004E000063EF820FC3EFE20043EF820FE3EFE20A4
:1004F000023EF820FE20F820023EFE20FE3EF820BC
:10050000043EFE20FC3EF820063EFE20FA3EF82087
:10051000083EFE20F63EF820083EFE20F63EF8207B
:10052000083EFE20F63EF820083EFE20F63EF8206B
:10053000083EFE20F63EF820083EFE20FA3EF82057
:10054000063EFE20FC3EF820043EFE20FE3EF82043
:10055000023EFE20F820FE20023EF820FE3EFE2055
:10056000043EF820FC3EFE20063EF820FA3EFE2027
:10057000083EF820F83EFE2008008511043EF820D1
:10058000063EFE200621F83EF820083EFE20F63EFC
:10059000F8200A3EFE20F43EF8200C3EFE20F23EFB
:1005A000F8200E3EFE20F13EF8200D3EFE20F33EE8
:1005B000F8200B3EFE20F53EF820093EFE20F63ED8
:1005C000F820083EFE20FA3EF820073EFE20FB3EC3
:1005D000F820063EFE20FC3EF820043EFE20FE3EB3
:1005E000F820013EFE20013EF820FE3EFE20033EA4
:1005F000F820FB3EFE20063EF820F83EFE20073E97
:10060000F820F73EFE20083EF820F63EFE20083E89
:10061000F820F73EFE20073EF820F83EFE20063E7A
:10062000F820FA3EFE20043EF820FD3EFE20013E6A
:10063000F820FE2008008511043EF820063EFE202A
:100640000621F83EF820083EFE20F63EF8200A3E3D
:10065000FE20F43EF8200B3EFE20F33EF8200C3E38
:10066000FE20F33EF8200B3EFE20F43EF8200A3E2A
:10067000FE20F63EF820083EFE20F83EF820063E1A
:10068000FE20FA3EF820043EFE20FD3EF820013E0A
:10069000FE20F820FE3EFE20043EF820FB3EFE2019
:1006A000073EF820F83EFE200A3EF820F73EFE20E6
:1006B0000B3EF820F63EFE200B3EF820F73EFE20D3
:1006C0000A3EF820F83EFE20073EF820FB3EFE20C2
:1006D000043EF820FE3EFE20F820013EFE20FD3EB6
:1006E000F820043EFE20FA3EF820053EFE20F93EAA
:1006F000F820063EFE20F93EF820053EFE20FA3E98
:10070000F820043EFE2008008511FA3EF820103E35
:10071000FE200621F23EF8200E3EFE20F43EF82098
:100720000C3EFE20F63EF8200A3EFE20F83EF82061
:10073000083EFE20FA3EF820063EFE20FC3EF82051
:10074000043EFE20FB3EF820033EFE20FC3EF82047
:10075000023EFE20FD3EF820013EFE20FE3EF82037
:10076000FE20FF3EF820FF3EFE20F820FE3EFE2049
:10077000013EF820FD3EFE20023EF820FC3EFE2019
:10078000033EF820FB3EFE2008008511FE3EF820C7
:10079000043EFE200621FA3EF820073EFE20F73EEA
:1007A000F8200A3EFE20F63EF8200C3EFE20F43EE5
:1007B000F8200E3EFE20F43EF8200D3EFE20F53ED1
:1007C000F8200C3EFE20F63EF8200A3EFE20F83EC1
:1007D000F820083EFE20FA3EF820053EFE20FD3EB1
:1007E000F820023EFE20FE3EF820FE20F820FE3ECD
:1007F000FE20F820FF3EFE20FF3EF820FE20FE3EB9
:10080000F820023EFE20FC3EF820043EFE20FA3E88
:10081000F820053EFE20F93EF820063EFE20FA3E76
:10082000F820043EFE20FC3EF820023EFE20FE3E64
:10083000F820FE20023EF820FD3EFE20053EF82076
:10084000FA3EFE20083EF820F83EFE200A3EF82040
:10085000F63EFE200C3EF820F53EFE200D3EF82030
:10086000F43EFE200C3EF820F63EFE200A3EF82024
:10087000F83EFE20083EF820FA3EFE20043EF82016
:10088000FD3EFE20013EF820FE2008008511063EB8
:10089000F820FE3EFE200621013EF820FD3EFE200F
:1008A000023EF820FC3EFE20023EF820FD3EFE20E7
:1008B000013EF820FE3EFE20F820013EFE20FD3ED7
:1008C000F820043EFE20FB3EF820073EFE20F83EC6
:1008D000F8200A3EFE20F73EF8200B3EFE20F63EB2
:1008E000F8200C3EFE20F63EF8200B3EFE20F73EA0
:1008F000F8200A3EFE20F83EF820073EFE20FB3E90
:10090000F820043EFE20FD3EF820013EFE20F820A7
:10091000FE3EFE20023EF820FC3EFE20043EF82073
:10092000FA3EFE20063EF820F83EFE20073EF82064
:10093000F73EFE20083EF820F63EFE20083EF82056
:10094000F73EFE20073EF820F83EFE20063EF82047
:10095000FA3EFE20043EF820FC3EFE2008008511F1
:10096000FA3EF820083EFE200621FA3EF820083E16
:10097000FE20FA3EF820083EFE20FA3EF820063E11
:10098000FE20FC3EF820043EFE20FE3EF820FE2025
:10099000023EF820FC3EFE20043EF820FA3EFE20F7
:1009A000063EF820F83EFE20083EF820F63EFE20E7
:1009B0000A3EF820F43EFE200C3EF820F23EFE20D7
:1009C0000C3EF820F63EFE20083EF820F63EFE20C3
:1009D000083EF820F83EFE20063EF820FA3EFE20B3
:1009E000043EF820FC3EFE20023EF820FE20F820C7
:1009F000023EFE20F820023EFE20F820FE20023EAD
:100A0000F820FE3EFE20043EF820FC3EFE20063E7E
:100A1000F820FA3EFE2008008511FA3EF820F73E45
:100A2000FE200621093EF820FA3EFE20063EF82070
:100A3000FD3EFE20033EF820033EFE20FD3EF82052
:100A4000063EFE20FA3EF8200B3EFE20F53EF82042
:100A5000083EFE20FA3EF820083EFE20FA3EF8202E
:100A6000073EFE20FC3EF820043EFE20FE3EF8201D
:100A7000013EFE20013EF820FD3EFE20043EF8200F
:100A8000F93EFE20073EF820F73EFE20083EF82003
:100A9000F53EFE20093EF820F53EFE20093EF820F6
:100AA000F63EFE20073EF820F93EFE20053EF820E7
:100AB000FC3EFE20023EF820FE2008008511F820B2
:100AC000043EFE200621FC3EF820023EFE20F820D7
:100AD000FE20F820023EFE20FC3EF820043EFE20D0
:100AE0008511FC3EF820FA3EFE200621063EF82045
:100AF000F83EFE200A3EF820F63EFE200A3EF82090
:100B0000F83EFE20063EF820FA3EFE200800851141
:100B1000083EF820043EFE200621FA3EF820033E5F
:100B2000FE20FB3EF820023EFE20FC3EF820013E67
:100B3000FE20FD3EF820FE20FE3EF820FF3EFE2077
:100B4000FF3EF820FE3EFE20F820FD3EFE20013E46
:100B5000F820FC3EFE2008008511F8207F3EFE2094
:100B60000621813EF8207B3EFE20853EF820773E20
:100B7000FE208511C93EF8202E3EFE200621D13EE2
:100B8000F8202E3EFE208511013EF820D23EFE20A8
:100B900006212D3EF820D23EFE208511403EF82051
:100BA000813EFE2006217B3EF820853EFE20773EDA
:100BB000F820893EFE2085116E3EF820523EFE2030
:100BC0000621AD3EF820543EFE2085117F3EF820E0
:100BD000523EFE200621AD3EF820543EFE208511F7
:100BE0006D3EF820813EFE2006217F3EF820853EA6
:100BF000FE207B3EF820893EFE208511373EF820FE
:100C0000D23EFE2006212F3EF820D23EFE20851146
:100C1000FF3EF8202E3EFE200621D33EF8202E3E39
:100C2000FE208511C03EF8207F3EFE200621853E35
:100C3000F8207B3EFE20893EF820773EFE2085117D
:100C4000923EF820AE3EFE200621533EF820AC3EF8
:100C5000FE208511813EF820AE3EFE200621533E47
:100C6000F820AC3EFE208511A33EF820CC3EFE20AD
:100C70000621343EF820CC3EFE2085113F3EF82070
:100C8000B53EFE2006214B3EF820B53EFE208511E4
:100C90004F3EF820A13EFE2006215F3EF820A13EF7
:100CA000FE2085115B3EF820953EFE2006216B3E1E
:100CB000F820953EFE208511603EF820953EFE20EE
:100CC00006216B3EF820953EFE2085115B3EF82004
:100CD000A03EFE200621603EF820A03EFE208511A9
:100CE000503EF820B53EFE2006214B3EF820B53E92
:100CF000FE208511403EF820CB3EFE200621353EE9
:100D0000F820CB3EFE208511313EF820DF3EFE204C
:100D10000621213EF820DF3EFE208511253EF820E9
:100D2000EB3EFE200621153EF820EB3EFE2085110D
:100D3000203EF820EC3EFE200621143EF820EC3E3A
:100D4000FE208511243EF820E03EFE200621203EB4
:100D5000F820E03EFE200800030113276E08FF0084
:100D60006F02F0006C08ED00342708008030EE00C0
:100D7000EF001430D3263A30EA00E4262030EA00AF
:100D8000E4260A30D32608008030EE00EF0014304D
:100D9000D326EA013B30E4261E30EA001F30E42669
:100DA0000A30D326080013276E08FF006F02F000F8
:100DB00003107C180314F60C0310FC180314F70C32
:100DC0006B08ED003427080013276E08FF006F0240
:100DD000F0007608EE007708EF006A081327FA01A2
:100DE0007C19FA037C18FA036E08F6070318FA0A4E
:100DF00003107A180314F60C7C10FA187C14FB010B
:100E0000FC19FB03FC18FB036F08F7070318FB0A28
:100E100003107B180314F70CFC10FB18FC146C086F
:100E2000ED00342708007D07C43E031C3C3EFE0055
:100E3000FC0DFC0D7C10FC10E13E03187C147E08B8
:100E4000F03E031C272F7E08D33E031CFC147E08B3
:100E500083169B001C141A08F60040309B071C14D4
:100E60001A08F70083120800F801F901FA01FB01E2
:100E70007F08F8208511FE200621ED0B402F080089
:100E80007608F8070318FA0A7C18FA037A0DFE00B0
:100E90007E0DFC39F81B0238781B01387F07EE0005
:100EA000F8207708F9070318FB0AFC18FB037B0DF1
:100EB000FE007E0DFC39F91B0238791B01387F07D3
:100EC0007007EF00FE203D2F83120313851B6E2F4A
:100ED000E80A083068060319772F6F2FE801051B11
:100EE0008D2FE90A1030690603197F2F8E2FF2012A
:100EF000F501F40A3C307406031D8C2FF401F20155
:100F0000F501F30A0C307306031D8D2FF301631CEA
:100F10008B2F63108C2F6314E801E9010B11FF3054
:100F20008100F20A32307206031DAE2FF201F50A7B
:100F30003C307506031DAE2FF501F40A3C307406F3
:100F4000031DAE2FF401F30A0C307306031DAE2F00
:100F5000F301631CAD2F6310AE2F63148B17202891
:02400E00703F01
:024200000000bc
:024202001b009f
:02420400350083
:024206004f0067
:0242080068004c
:02420a007f0033
:02420c0096001a
:02420e00ab0003
:02421000be00ee
:02421200ce00dc
:02421400dd00cb
:02421600e900bd
:02421800f300b1
:02421a00f900a9
:02421c00fe00a2
:02421e00ff009f
:02422000fe009e
:02422200f900a1
:02422400f300a5
:02422600e900ad
:02422800dd00b7
:02422a00ce00c4
:02422c00be00d2
:02422e00ab00e3
:024230009600f6
:024232007f000b
:02423400680020
:024236004f0037
:0242380035004f
:02423a001b0067
:02423c00000080
:02423e00e50099
:02424000cb00b1
:02424200b100c9
:024244009800e0
:024246008000f6
:024248006a000a
:02424a0055001d
:02424c0042002e
:02424e0032003c
:02425000230049
:02425200170053
:024254000d005b
:0242560007005f
:02425800020062
:02425a00010061
:02425c0002005e
:02425e00070057
:024260000d004f
:02426200170043
:02426400230035
:02426600320024
:02426800420012
:02426a005500fd
:02426c006a00e6
:02426e008000ce
:024270009800b4
:02427200b10099
:02427400cb007d
:02427600e50061
:02427800000044
:02427a001b0027
:02427c0035000b
:02427e004f00ef
:02428000ff003d
:02428200fe003c
:02428400f9003f
:02428600f30043
:02428800e9004b
:02428a00dd0055
:02428c00ce0062
:02428e00be0070
:02429000ab0081
:02429200960094
:024294008000a8
:024296006800be
:024298004f00d5
:02429a003500ed
:02429c001b0005
:02429e0000001e
:0242a000e50037
:0242a200cb004f
:0242a400b10067
:0242a60098007e
:0242a800810093
:0242aa006a00a8
:0242ac005500bb
:0242ae004200cc
:0242b0003200da
:0242b2002300e7
:0242b4001700f1
:0242b6000d00f9
:0242b8000700fd
:0242ba00020000
:0242bc000100ff
:0242be000200fc
:0242c0000700f5
:0242c2000d00ed
:0242c4001700e1
:0242c6002300d3
:0242c8003200c2
:0242ca004200b0
:0242cc0055009b
:0242ce006a0084
:0242d00080006c
:0242d200980052
:0242d400b10037
:0242d600cb001b
:0242d800e500ff
:0242da000000e2
:0242dc001b00c5
:0242de003500a9
:0242e0004f008d
:0242e200680072
:0242e400800058
:0242e600960040
:0242e800ab0029
:0242ea00be0014
:0242ec00ce0002
:0242ee00dd00f1
:0242f000e900e3
:0242f200f300d7
:0242f400f900cf
:0242f600fe00c8
:0242f800ff00c5
:0242fa00fe00c4
:0242fc00f900c7
:0242fe00f300cb
:00000001FF
